:1000030041000300410004004100000041000100E1
:0400130041000200A6
:030023000205B91A
:1005B900C0E0C083C082C0D075D010309828C298DE
:1005C900900001E02401FFE433FEA3E06F7001EE27
:1005D9006014900001E0FF04F074052FF582E43403
:1005E90000F583E599F0309927C299900004E0FF5E
:1005F900900003E06F6013A3E004F074052FF58207
:10060900E43401F583E0F59980069000007401F067
:09061900D0D0D082D083D0E032B1
:10072D007FB07E04120622C2AFE4900003F0A3F066
:10073D0090000004F0E4A3F0A3F0C29FD29EC29DEE
:0D074D00D29CC299C298D2ACC2BCD2AF22DD
:10062200C2AFC299E4900003F0A3F090000004F07E
:10063200C28EC2AB43878053890F438920E4FCFDFD
:100642007BC0FAF9F8120382A804A905AA06AB072F
:100652007F007E1B7DB77C00120667EFF404F58DE8
:05066200D28ED2AF2290
:1006EE008F3B1207F0C3E49FFF74019400FED3EF1B
:1006FE009402EE940050037FFF22C2AF900003E0FD
:10070E00FF04F074052FF582E43401F583E53BF028
:0F071E00900000E06004E4F0D299D2AF7F002297
:1007AD001207E3EF70057EFF7FFF22C2AF900002BC
:1007BD00E0FF04F074052FF582E43400F583E0FFCB
:0407CD00D2AF7E0029
:0107D1002205
:0D07E300900002E0FF900001E0C39FFF22A4
:0D07F000900004E0FF900003E0C39FFF2293
:10075A000A000A48692D74726F6E69630A0025637C
:10076A000A00596F7520707265737365642025637A
:0C077A000A00546869732069732E0A009D
:0B07FD001207ADEFF47002EEF460F59F
:0108080022CD
:020786008F38AA
:10078800AF381206EEEF601AE4F539F53AC3E53AE8
:1007980094E8E539940350E8053AE53A70020539DA
:0407A80080EBAF38FB
:0107AC00222A
:1006AB0012072D7FB07E041206227BFF7A07795A40
:0F06BB0075270A1200887BFF7A07795C12008886
:1006CA007BFF7A07796875270A1200881207D28F8A
:1006DA0022E52204F5237BFF7A07796CF5271200BD
:0306EA008880DD28
:0106ED0022EA
:0300000002052DC9
:0C052D00787FE4F6D8FD75813B02057470
:10038200E88FF0A4CC8BF0A42CFCE98EF0A42CFC1A
:100392008AF0EDA42CFCEA8EF0A4CDA8F08BF0A498
:1003A2002DCC3825F0FDE98FF0A42CCD35F0FCEBF7
:1003B2008EF0A4FEA9F0EB8FF0A4CFC5F02ECD39BC
:0F03C200FEE43CFCEAA42DCE35F0FDE43CFC2229
:10066700C2D5E830E70FB2D5E4C39BFBE49AFAE4BE
:1006770099F9E498F8EC30E717B2D512069D120401
:1006870065E4C39BFBE49AFAE499F9E498F88003DC
:1006970012046530D50DE4C39FFFE49EFEE49DFD83
:0406A700E49CFC22B1
:10002600E5332427F8E605332278243007027827BB
:10003600E475F0011204F70203D12000EB7F2ED203
:10004600008018EF540F2490D43440D4FF30040BB2
:10005600EF24BFB41A0050032461FFE53460021593
:10006600340537E5377002053630070D7824E47518
:10007600F0011204F7EF0204170207867403D20791
:100086008003E4C207F5338B248A258926E4F534F8
:10009600F536F537E53460077F2012006180F57587
:1000A60035FFC201C200C202C203C205C206C208AF
:1000B60012002FFF700D3007057F00120072AF3758
:1000C600AE3622B4255FC2D5C20412002FFF24D05B
:1000D600B40A00501A75F00A783430D50508B6FF10
:1000E6000106C6A426F620D5047002D20380D924C0
:1000F600CFB41A00EF5004C2E5D204020272D20154
:1001060080C6D20080C0D20280BCD2D580BAD205C9
:1001160080B47F201200612002077401B5340040CC
:10012600F1120026FF12006102009AD208D2068060
:1001360095120026FB120026FA120026F94A4B7089
:100146000679437A037BFF20022EE534602A7E007F
:100156008E827583001203EA60060EEE653570F036
:10016600C2D5EBC0E0EAC0E0E9C0E0EE1202B9D0C9
:10017600E0F9D0E0FAD0E0FB1203D1FF60AAEBC0B1
:10018600E0EAC0E0E9C0E0120061D0E02401F9D065
:10019600E03400FAD0E0FBE5350460DCD535D980E3
:1001A600877BFF7A0279B5D202809C79108002792A
:1001B60008C206C2088008D2D5790A8004790AC224
:1001C600D5E535047002F535E4FAFDFEFF1200268A
:1001D600FC7B08200113120026FD7B1030000A125A
:1001E6000026FE120026FF7B20EC3382D592D550E6
:1001F60013C3E43000069FFFE49EFEE42001039D46
:10020600FDE49CFCE4CBF8C201EC700CCFCECDCC67
:10021600E824F8F870F38017C3EF33FFEE33FEEDF2
:1002260033FDEC33FCEB33FB994002FB0FD8E9EBD3
:10023600300105F8D0E0C448B201C0E00AEC4D4EEA
:100246004F78207B0070C2EAB5350040BCC0E01292
:1002560002BBD0F0D0E0200104C4C0E0C4B201C0AB
:10026600F012004AD0F0D5F0EB02009A1205070111
:10027600375301B15801084C01044201B54F01BD85
:0F0286004401BD49011D4301C35501A74601A70E
:100295004501A747036350010C2D01102E01332B97
:1002A500011423013120034C2A00CC480000012B06
:1002B5003F3F3F00790AA2D5200314300509B91044
:1002C500020404B9080104A2D52006025001042045
:1002D50002689202B534005034C0E07F2030031923
:1002E5007F30A20272067205500F120312C202C2BB
:1002F50006C205C2087F30800F300503E9C0E01251
:100305000061300503D0E0F9D0E0B534CC300517F5
:100315007F30B9100C1200617F583004077F788058
:1003250003B908031200613002057F2D0200617FC9
:10033500202008F87F2B2006F322920280CF286E1A
:10034500756C6C2900D2011200263001F8C20178C3
:100355003430D50108F60200CC2D5043495812001F
:10036500262403B405004001E490035E9312005275
:0D037500743A120052D2037534040201B133
:1007D20010090B1207FDBF0D027F0A020786AF0840
:0107E20022F4
:100539000206ABE493A3F8E493A34003F68001F227
:1005490008DFF48029E493A3F85407240CC8C333C3
:10055900C4540F4420C8834004F456800146F6DF92
:10056900E4800B0102040810204080900003E47E1F
:10057900019360BCA3FF543F30E509541FFEE49387
:10058900A360010ECF54C025E060A840B8E493A34E
:10059900FAE493A3F8E493A3C8C582C8CAC583CA79
:1005A900F0A3C8C582C8CAC583CADFE9DEE780BE31
:0100170000E8
:1003D100BB010689828A83E0225002E722BBFE022A
:0903E100E32289828A83E493225D
:1003EA00BB010CE58229F582E5833AF583E02250C8
:1003FA0006E92582F8E622BBFE06E92582F8E22212
:0D040A00E58229F582E5833AF583E493222B
:10041700BB010689828A83F0225002F722BBFE01C4
:02042700F322BE
:1004290075F008758200EF2FFFEE33FECD33CDCC8A
:1004390033CCC58233C5829BED9AEC99E58298400D
:100449000CF582EE9BFEED9AFDEC99FC0FD5F0D6EA
:10045900E4CEFBE4CDFAE4CCF9A88222B800C1B914
:100469000059BA002DEC8BF084CFCECDFCE5F0CB52
:10047900F97818EF2FFFEE33FEED33FDEC33FCEB8B
:1004890033FB10D703994004EB99FB0FD8E5E4F946
:10049900FA227818EF2FFFEE33FEED33FDEC33FC33
:1004A900C933C910D7059BE99A4007EC9BFCE99A27
:1004B900F90FD8E0E4C9FAE4CCFB2275F010EF2F6C
:1004C900FFEE33FEED33FDCC33CCC833C810D7076C
:1004D9009BEC9AE899400AED9BFDEC9AFCE899F8A7
:0E04E9000FD5F0DAE4CDFBE4CCFAE4C8F9223A
:1004F700FAE6FB0808E6F925F0F618E6CA3AF62206
:10050700D083D082F8E4937012740193700DA3A383
:1005170093F8740193F5828883E473740293686097
:06052700EFA3A3A380DF97
:00000001FF
